:0200000480007A
:10000000B72F0000938F0F8073900F3015A8130047
:100010000000130000001300000013000000130094
:100020000000130000001300000013000000130084
:100030000000130000001300000013000000010086
:10004000970200009382020C73905230814001416C
:100050008141014281420143814301448144014580
:100060008145014681460147814701488148014950
:100070008149014A814A014B814B014C814C014D20
:10008000814D014E814E014F814F971102009381A6
:1000900061C9170502001305E54A9795030093858A
:1000A000257201461122170502001305253F970509
:1000B00002009385E5460146C52817A503001305F0
:1000C000657097B503009385A56F37B6ABAB130684
:1000D000B6BAD92817B103001301C16EEF60401AF8
:1000E000860293D21200F512638802008242110147
:1000F0006F00001073002030824211017300203025
:10010000711116C0F3222034E3CC02FC82421101AB
:10011000130141F806C20AC40EC612C816CA1ACC88
:100120001ECE22D026D22AD42ED632D836DA3ADCC7
:100130003EDEC2C0C6C2CAC4CEC6D2C8D6CADACC97
:10014000DECEE2D0E6D2EAD4EED6F2D8F6DAFADCA7
:10015000FEDE73252034F32510340A8601A07310C7
:10016000153492402241B2414242D2426243F243AC
:10017000025492542255B2554256D2566257F25703
:10018000064896482649B649464AD64A664BF64B33
:10019000065C965C265DB65D465ED65E665FF65F83
:1001A0001301C1077300203010C16374B50011053D
:1001B000E5BF828000000000000000000000000099
:1001C000000000000000000000000000000000002F
:1001D000000000000000000000000000000000001F
:1001E000000000000000000000000000000000000F
:1001F000197106C00AC20EC412C616C81ACA1ECC8D
:1002000022CE26D02AD22ED432D636D83ADA3EDCC6
:1002100042DEC6C0CAC2CEC4D2C6D6C8DACADECC96
:10022000E2CEE6D0EAD2EED4F2D6F6D8FADAFEDCA6
:100230009702020083A2C22923A02200F3221034D5
:1002400096DEEF00002B1701020003216128024116
:10025000F65273901234B72200009382028873A082
:10026000023082403242C2425243E24372448254DC
:100270001255A2553256C2565257E2577258864806
:100280001649A649364AC64A564BE64B764C865C1A
:10029000165DA65D365EC65E565FE65F0961730059
:1002A0002030970202009382E22923A0120023A2A9
:1002B000220023A4320023A6420023A8520023AA2E
:1002C000620023AC720023AE820023A0920223A21C
:1002D000A20223A4B20223A6C20223A8D20223AA06
:1002E000E20223ACF20223AE020323A0120523A2F2
:1002F000220523A4320523A6420523A8520523AADA
:10030000620523AC720523AE820523A0920723A2C7
:10031000A20723A4B20723A6C20723A8D20723AAB1
:10032000E20723ACF207EF40B04B170102000321B4
:10033000211A0241F65273901234B72200009382C0
:10034000028873A0023082403242C2425243E243EA
:10035000724482541255A2553256C2565257E25731
:10036000725886481649A649364AC64A564BE64B45
:10037000764C865C165DA65D365EC65E565FE65FB1
:10038000096173002030970202009382A21B83A0B0
:10039000020003A1420083A1820003A2C20083A243
:1003A000020103A3420183A3820103A4C20183A427
:1003B000020203A5420283A5820203A6C20283A60B
:1003C000020303A7420383A7820303A8C20383A8EF
:1003D000020403A9420483A9820403AAC20483AAD3
:1003E000020503AB420583AB820503ACC20583ACB7
:1003F000020603AD420683AD820603AEC20683AE9B
:10040000020703AFC20983AF820782807370043092
:10041000197106C00AC20EC412C616C81ACA1ECC6A
:1004200022CE26D02AD22ED432D636D83ADA3EDCA4
:1004300042DEC6C0CAC2CEC4D2C6D6C8DACADECC74
:10044000E2CEE6D0EAD2EED4F2D6F6D8FADAFEDC84
:100450009702020083A2C20723A0220086DEEF20BB
:100460002053170102000321A1060241F6527390A6
:100470001234B72200009382028873A002308240B7
:100480003242C2425243E243724482541255A25550
:100490003256C2565257E257725886481649A649F4
:1004A000364AC64A564BE64B764C865C165DA65DD0
:1004B000365EC65E565FE65F09617300203073707A
:1004C000043001A07310453082807325403073F0F2
:1004D00043308280970700009387A7FE232EB5FE46
:1004E0002322C5FA232635F82320F5F8130505F84D
:1004F0008280411106C6EF40D02BEF10502F01E54E
:10050000B24041018280B24041016F2060489307B0
:1005100085007D575CC118C55CC51CC9232005003A
:1005200082802328050082805C41DCC1984798C501
:1005300098474CC38CC788C91C4185071CC1828061
:100540009041FD57130785006314F60039A83E87D4
:100550005C439443E37DD6FEDCC18CC798C54CC395
:1005600088C91C4185071CC1828018495C43EDB7CE
:10057000584114451C4914C71845544154C3D84325
:100580006314A7001845D8C32328050088437D15A8
:1005900088C382803041AE8701CE4C455841B29528
:1005A0004CC563E4E5000C414CC53E856F30F0441A
:1005B0008280411122C406C62A8426C2EF207036EA
:1005C0003C44635BF0025C5085CB9304440209A871
:1005D0003C44FD173CC43C446350F0025C5089CF5E
:1005E0002685EF20807C6DD5EF20701C3C44FD17E4
:1005F0003CC43C44E344F0FEFD573CC4EF20B0341F
:10060000EF2030327C40635BF0021C4885CB9304C2
:10061000040109A87C40FD177CC07C406350F002B7
:100620001C4889CF2685EF2040786DD5EF20301803
:100630007C40FD177CC07C40E344F0FEFD577CC04D
:100640002244B240924441016F20F02F29C541114C
:1006500022C426C22A8406C6AE84EF20902C3440E1
:100660005C5C1840232C0402B387F6027D5670C0F0
:1006700018C430C4B386D740BA9736975CC058C404
:1006800091EC1C489DE3EF20102CB2402244924490
:100690000545410182807370043001A013050401F7
:1006A000BD3513054402A535F9BF13050401EF203C
:1006B000C06F8547E319F5FC913BF1B701E5737015
:1006C000043001A0011126CA4AC84EC606CE22CC6B
:1006D000B2892E89AA84A5C53305B502130555052F
:1006E000EF3070192A8435C1930745051CC144DCDD
:1006F00023202405EF20F02234405C5C18407D5616
:10070000B387F602232C040270C018C430C413054A
:100710000401B386D740BA9736975CC058C4C53B2E
:1007200013054402ED33EF201022230834052285FF
:10073000F2406244D2444249B249056182801305C5
:100740004005EF3050132A8401E57370043001A096
:1007500000C071BF01E57370043001A06375B5007E
:100760007370043001A0411122C409462E848145D2
:1007700006C6A93711C500DDB2402244410182807E
:100780007370043001A05D7186C6A2C4A6C2CAC03F
:100790004EDE52DC56DA5AD85ED632C6630A051CE3
:1007A0006382051C89476399F600585D8547630598
:1007B000F7007370043001A03689AE842A84EF20DC
:1007C000900111E5B24781C77370043001A0EF209A
:1007D0005015185C5C5C014B894BFD59130A0401F0
:1007E000930A44026365F70C63077919B247638182
:1007F000072463150B002808EF20406EEF20B0148B
:10080000EF10A075EF20F0117C4063943701232294
:1008100004043C446394370123240404EF20B01201
:100820006C002808EF20A06D631E051EEF20700FDE
:10083000185C5C5C630CF70AEF20F010EF20700E80
:100840003C44634FF00039A85685EF20005619C18B
:10085000EF20E0753C44FD173CC43C446354F00079
:100860005C50FDF323243405EF20F00DEF20700BD6
:100870007C40634FF00039A85285EF20005319C126
:10088000EF20E0727C40FD177CC07C406354F00098
:100890001C48FDF323223405EF20F00AEF10F0107E
:1008A000054BEF201008185C5C5CE37FF7F23040EA
:1008B0006305060C631F09120844A685EF30F01388
:1008C0001C4434405840B6971CC463EAE70A1C5CD9
:1008D00014405850850714C41CDC5DC7130544023E
:1008E000EF20A04C85476311F50AC9A8EF20B00599
:1008F000B2455285EF20202DEF20B0023C44634FDB
:10090000F00039A85685EF20404A19C1EF20206A2F
:100910003C44FD173CC43C446354F0005C50FDF380
:1009200023243405EF203002EF20A07F7C40634F6A
:10093000F00039A85285EF20404719C1EF20206709
:100940007C40FD177CC07C406354F0001C48FDF3E4
:1009500023223405EF20207FEF10300531F17D3464
:10096000054B81B73C41E38F07E27370043001A06F
:100970007370043001A0304021E61C4085C71C5C28
:10098000585085071CDC39FBEF20E07B0545B6405D
:10099000264496440649F259625AD25A425BB25BE7
:1009A000616182804840EF20206F1C5C58502322F8
:1009B000040085071CDCE31307F279D5813CE9B715
:1009C0004844A685EF3070033C4058441440B307B8
:1009D000F0403E9758C4637CD7025840BA975CC435
:1009E00009475C506306E902185C050718DCC9DF9B
:1009F000F5B54844A685EF3050003C4058441440BB
:100A0000B307F0403E9758C4E37CD7FCF9B75C507D
:100A1000185C79DB185C7D1718DC185C050718DC9E
:100A2000A5D76DBD22857136EF102078014585B7B9
:100A3000EF2060710145A1BF411126C2AA841305B0
:100A4000400522C406C6EF3000632A8415CD232C4E
:100A50000502FD577CC10547410558DC3CC42322F3
:100A60000400232004002324040023260400232060
:100A7000040423089404613C13054402493C814664
:100A800001468145228501332285B24022449244A9
:100A9000410182800DC5411122C426C206C64AC04A
:100AA000032945002A84EF2040528144630CA900A9
:100AB000B2402244268502499244410182807370EB
:100AC000043001A05C448544FD175CC4F5F3814605
:100AD0000146814522854539E1BF397106DE22DCB8
:100AE00026DA4AD84ED652D432C635CD8149DDC138
:100AF0003689AE842A84130A05012DA0EF20A06454
:100B0000EF2020626C002808EF20603F31E1EF20E9
:100B10004061185C5C5C6305F702EF20C062EF2067
:100B200080628549EF20E05F185C5C5C6360F704DD
:100B3000B24799CFE39409FC2808EF20203A7DBF03
:100B4000EF206060B2455285EF20E007C130C1BFA1
:100B5000EF20605FF2506254D2544259B259225A87
:100B60000145216182807370043001A0304015EE90
:100B70001C4095C71C5C585085071CDC39E7EF20EA
:100B8000805CF2506254D2544259B259225A0545FF
:100B9000216182803C41A9DF7370043001A048408C
:100BA000EF20804F23220400F1B7631909020844A3
:100BB000A685EF3080641C4434405840B6971CC46E
:100BC000E3EAE7FA1C401CC475B713054402EF20A2
:100BD000C01D8547E315F5FA153855B74844A68575
:100BE000EF30A0613C4058441440B307F0403E97BA
:100BF00058C46375D7005840BA975CC48947E31B53
:100C0000F9F61C5CA5DB1C5CFD171CDCA5B7397173
:100C100006DE22DC26DA4AD84ED652D432C663012A
:100C2000050E81446388050CB6892E892A84130A2F
:100C3000450231A0EF202051EF20E0508544EF2005
:100C4000404E1C5CBDE3B24795CF8DC8EF20A04F4E
:100C5000EF20204D6C002808EF20602A05E5EF20EA
:100C6000404C1C5CE1FBEF20004E1C409DC7B24590
:100C70005285EF105075EFF06FF97DBF2808EF2017
:100C8000E025E9B7EF20204CF2506254D25442598B
:100C9000B259225A014521618280EF2080484840A4
:100CA000EF206035EF20204AD9B73040444409CEC8
:100CB0005840B387C4005CC463E4E7001C405CC4D4
:100CC0004C444A85EF306053639F09021C5C184016
:100CD000FD171CDC01E7EF20804B48C01C489DC776
:100CE00013050401EF20600C85476311F502EFF056
:100CF000EFF129A83C41E38907F27370043001A0A9
:100D00007370043001A05C5044C481EFEF20A04315
:100D1000F2506254D2544259B259225A05452161C7
:100D2000828013054402EF2040086DD1C9B725C168
:100D3000B1C9011122CC26CA4AC852C406CE4EC639
:100D40008947B68432892E8A2A846399F600585DD1
:100D500085476301F7067370043001A0EFF0EFF6EA
:100D6000185C5C5CAA896367F70281444E85EFF0EA
:100D70006FF5F240624426854249D244B249224A84
:100D8000056182803C41D5D77370043001A0737037
:100D9000043001A0304049E21C40DDCB1C5C7D5793
:100DA00085071CDC3C446388E7083C448544850790
:100DB0003CC46DBFEFF06FF1185C5C5CAA89636D99
:100DC000F702304071DA4844D285EF3000433C40AE
:100DD00058441440B307F0403E9758C46375D70099
:100DE0005840BA975CC48947E39AF4FA1C5CDDD793
:100DF0001C5CFD171CDC5DB7304059DE4844D285D1
:100E0000EF30A03F3C4058441440B307F0403E97B9
:100E100058C4E367D7FCD9BFDDF40844D285EF306E
:100E2000C03D1C4434405840B6971CC4E3E8E7F684
:100E30001C401CC4A5B75C5085448DDB13054402DF
:100E4000EF10B07605D5E30309F22320990039BFEE
:100E50004840EF2060242322040089B731CD3C4173
:100E600081C77370043001A01C41B1CB011122CCA9
:100E700026CA2A844AC84EC606CE2E89EFF0EFE471
:100E8000185C5C5CAA898144637DF7001C5C7D571B
:100E900085071CDC3C446389E7023C4485448507A4
:100EA0003CC44E85EFF00FE2F24062442685424991
:100EB000D244B249056182807370043001A05C4164
:100EC000D5D77370043001A05C5099E38544D1BF3D
:100ED00013054402EF10706D75D9E30909FE8547CB
:100EE0002320F900E5B7397106DE22DC26DA4AD87C
:100EF0004ED652D456D232C66302051C638A051AF6
:100F0000B68AAE892A84EF20000D11E5B24781C769
:100F10007370043001A0EF20C0201C5C63920714A2
:100F2000B247638E070A2808EF10507BFD5413095F
:100F30004402130A0401EF200021EF100002EF2009
:100F4000401E7C4063949700232204043C44639435
:100F5000970023240404EF20001F6C002808EF10E2
:100F6000107A63130518EF20C01B1C5CADCFEF2077
:100F7000801DEF20001B3C44634FF00039A84A85D8
:100F8000EF10B06219C1EF2080023C44FD173CC451
:100F90003C446354F0005C50FDF324C4EF20A01ADD
:100FA000EF2020187C40634FF00039A85285EF10E5
:100FB000D05F19C1EF10B07F7C40FD177CC07C4032
:100FC0006354F0001C48FDF364C0EF20C017EF101D
:100FD000C01DEF2000151C5CC1E7B247A9FFEF2040
:100FE0008016014555A0EF2000161C40DDC7B24514
:100FF0004A85EF10503DEF20C0123C44634FF00093
:1010000039A84A85EF10705A19C1EF10507A3C4444
:10101000FD173CC43C446354F0005C50FDF324C411
:10102000EF206012EF20E00F7C40634FF00039A802
:101030005285EF10905719C1EF1070777C40FD1763
:101040007CC07C406354F0001C48FDF364C0EF207A
:10105000800FEF10801531C9EF20A00C1C5CB5DFAC
:10106000CE8522854444EFF0EFD2639C0A041C5CD9
:101070001840FD171CDC01E7EF20601148C01C4838
:10108000A1EFEF20400C0545F2506254D254425972
:10109000B259225A925A21618280EF20800848403A
:1010A000EF107075EF20200A99B7EFF02FB66DB7EB
:1010B0003C41E38707E47370043001A0737004308F
:1010C00001A05C5044C4D5DF13054402EF10F04D7D
:1010D0004DD9EFF0AFB375B713050401EF10F04C25
:1010E0008547E310F5FAF5B72285EFF08FCCEF10C6
:1010F000C00B014551BF1DC9411122C44AC006C6DB
:1011000026C244412E892A84EF10306C6383A402E6
:1011100081464A8681452285F93385476300F50279
:10112000B2402244924402494101828073700430EB
:1011300001A05C44054585075CC4DDB75C448507B8
:101140005CC4F9BF15CDADC9011122CC26CA4AC86D
:101150004EC652C42A8406CE3289AE89EFF0EFB66D
:101160001C5C2A8A814485E35285EFF0AFB5F240DA
:10117000624426854249D244B249224A05618280AE
:101180007370043001A0304001CE4C445C40B295F5
:101190004CC463E4F5000C404CC44E85EF30E005D0
:1011A0001C5C7D57FD171CDC7C40638CE7007C4099
:1011B000854485077CC04DBF3C41D9D7737004304E
:1011C00001A01C4899E3854445B713050401EF10BD
:1011D000D03D75D9E30909FE85472320F900E5B71D
:1011E00021C93C41A1CDA1CB011122CC26CA4AC8BC
:1011F00052C42A8406CE4EC62E8AEFF00FAD1C5C78
:101200002A89814491CB8329C400D2852285EFF0BD
:101210006FB88544232634014A85EFF0AFAAF24027
:10122000624426854249D244B249224A05618280FD
:101230007370043001A07370043001A0EDDF73708F
:10124000043001A001E57370043001A0411122C4F3
:101250002A8406C6EF10F06C005CEF10D06EB2402E
:10126000228522444101828001E57370043001A08F
:10127000411106C622C42A84EF10B06A1C5C405C8F
:101280001D8CEF10506C2285B240224441018280B7
:1012900019C1085D82807370043001A01DCD97874D
:1012A00003009387274ED843630CE502D847630CAD
:1012B000E504D84B6307E504D84F6302E504D8532F
:1012C000630DE502D8576308E502D85B6303E502C6
:1012D000D85F630EE5006F20306C7370043001A09E
:1012E00001470E07BA9723A007006F20F06A1D4739
:1012F000CDBF1947FDB71547EDB71147DDB70D470E
:10130000CDB70947F9BF0547E9BF684582806CC57D
:10131000828003450505828009C5085D13351500E7
:1013200082807370043001A019C51C5D485D1D8D5D
:101330001335150082807370043001A09787030075
:1013400093874744984305C3984705C7984B05C7FB
:10135000984F05C7985305C7985705C7985B15C799
:10136000985F15C3828001470E07BA978CC3C8C324
:1013700082800547D5BF0947C5BF0D47F5B711475F
:10138000E5B71547D5B71D47C5B71947F1BF9787CB
:1013900003009387273FD8436308E502D847630BD0
:1013A000E502D84B630AE502D84F6309E502D8533A
:1013B0006308E502D8576307E502D85B6308E502D6
:1013C000D85F6303A702828001470E07BA9723A064
:1013D000070082800547D5BF0947C5BF0D47F5B750
:1013E0001147E5B71547D5B71D47C5B71947F1BF31
:1013F000411122C426C24AC02A8406C6AE8432895C
:10140000EF1030527840FD576314F7002322040494
:101410003844FD576314F70023240404EF10B0523E
:101420001C5C99E74A86A68513054402EF10B00CB0
:10143000EF10304F3C44635BF0025C5085CB93046B
:10144000440209A83C44FD173CC43C446350F002EC
:101450005C5089CF2685EF1050156DD5EF103035D3
:101460003C44FD173CC43C44E344F0FEFD573CC4FF
:10147000EF10704DEF10F04A7C40635BF0021C48A7
:1014800085CB9304040109A87C40FD177CC07C40F7
:101490006350F0021C4889CF2685EF1010116DD5DE
:1014A000EF10F0307C40FD177CC07C40E344F0FE40
:1014B000FD577CC02244B2409244024941016F1062
:1014C000904805C579714ECE52CC06D63E8A22D4BC
:1014D00026D24AD056CA5AC85EC662C4A547BA893F
:1014E00063F8E7007370043001A07370043001A04A
:1014F000AA8AAE843289B68B428B6309082213050F
:101500000006EF2050372A84630D05200A0923289E
:1015100065034A869305500A5A85EF20105C03C77D
:1015200004001C587119230AE40203C704003E9901
:101530001379C9FF79C783C71400A30AF40283C7CC
:101540001400E1C383C72400230BF40283C72400E3
:10155000CDCB83C73400A30BF40283C73400D5C3BB
:1015600083C74400230CF40283C74400D9CB83C74C
:101570005400A30CF40283C75400C1C783C764009E
:10158000230DF40283C76400ADCF83C77400A30D9D
:10159000F40283C77400B5C783C78400230EF40226
:1015A00083C78400B9CF83C79400A30EF40283C716
:1015B0009400A1CB83C7A400230FF40283C7A40027
:1015C000A9C383C7B400A30FF40283C7B40095CBAB
:1015D00083C7C4002300F40483C7C4009DC383C72A
:1015E000D400A300F40483C7D40081CF83C7E400F0
:1015F0002301F40483C7E40089C783C7F400A3016F
:10160000F404130B44005A85A30104042326340375
:1016100023283405232A0404EFE0BFF013058401D6
:10162000EFE03FF0A947B3873741232C040400C8FB
:101630001CCC40D023220404232E04045E86D685CD
:101640004A85EFE03FE908C063040A0023208A00CE
:101650007370043017F901001309C9E583270900E5
:1016600097F401009384C4E691C798409C407C4362
:1016700085077CC317F70100130787E41C43850720
:1016800097F6010023AEF6E29C40D5CB83270900F4
:1016900017FA0100130ACAF289EB9C40DC5763E693
:1016A000F90097F7010023A587E297F701009387D8
:1016B00067DF984397F60100938606E05C549442F6
:1016C000050717F60100232FE6DC38C463F6F600A1
:1016D00017F701002322F7DE5147B387E702DA85C7
:1016E0003305FA00EFE05FE48327090081C79C40DF
:1016F000FC43BDE383270900054499C79C40DC57A0
:1017000063F43701EFE09FD02285B2502254925407
:101710000259F249624AD24A424BB24B224C4561CD
:1017200082805A85EF2050277D54F9BF131526007B
:10173000EF2070142A8BE31405DC7D54F1B797F782
:10174000010023A787D8184385476301F70217FADA
:101750000100130AEAE691BF984094407C43FD17CC
:101760007CC3FC42C1FB7360043069B7814A17FA3D
:101770000100130AEAE4514CA94B33858A03850A18
:101780005295EFE0DFD8E39A7AFF97FB0100938B45
:10179000ABEF5E85EFE0BFD797FA0100938A0AF0BE
:1017A0005685EFE0DFD617F50100130565F0EFE091
:1017B0001FD617F501001305E5F0EFE05FD517F52B
:1017C0000100130565F1EFE09FD497F7010023AF07
:1017D00077CF97F7010023A957CFC1BD411122C48C
:1017E00006C626C24AC02A847370043097F40100EA
:1017F000938444CC9C40F9E311E497F7010093876C
:1018000027CD8043130944004A85EFE07FD61C545E
:1018100089C713058401EFE0BFD5CA8517F501001C
:10182000130545EAEFE05FD097F70100938787C97A
:10183000984397F701009387E7C69C43050797F6FF
:10184000010023A1E6C89840850797F6010023AB65
:10185000F6C401CB97F70100938787C79843784375
:1018600049EF9C40B1C797F70100938767C698433B
:10187000630F870873700430984039EB17F7010045
:101880001307C7C414439442A5E27D5797F601009D
:1018900023A8E6C0984009CF9843784311CB9843DA
:1018A00094437C43FD177CC3FC4299E3736004308E
:1018B000B2402244924402494101828097F70100DC
:1018C000938707C198439C437C4385077CC32DB70E
:1018D00094439843F8420507F8C217F7010013072D
:1018E000E7BE14439442D5D218435847584758434B
:1018F00097F6010023A6E6BA71BF984394437C4350
:10190000FD177CC3FC42B1FF7360043099BF97F7A9
:1019100001009387A7B89C4381C77370043001A06E
:101920002244B2409244024941016FE03FAE41C5BA
:1019300017F701001307C7B914438147638BA60645
:10194000411106C622C426C27370043097F6010006
:10195000938646B69C4291C710431C437C42850740
:101960007CC29C42AA84404981C71C43FC43B9E71E
:1019700097F70100938787B59C43638B870497F79C
:101980000100938767B49C436384870497F7010041
:10199000938787D46309F40297F70100938787D26E
:1019A0006301F4028547B240224492443E854101DE
:1019B00082803E8582807370043001A0EF40B001C8
:1019C00045BF9147CDB79C5493B717008907E1BF36
:1019D0008947D1BF7370043097F70100938787ADB3
:1019E000984309EF15C59C43485581CB97F70100F3
:1019F000938707AE9843784315E3828017F7010079
:101A0000130707AD14431843F8420507F8C261FDF8
:101A100017F701001307C7AB0843F1B79843944386
:101A20007C43FD177CC3FC42E9FB73600430828079
:101A3000411122C42A8406C6EFE03FA911E497F7BA
:101A400001009387E7A880434054EFE0BFA7B2406E
:101A50002285224441018280A54763F5B700737057
:101A6000043001A0011122CC06CE26CA4AC84EC6B7
:101A700052C42A847370043017F90100130989A332
:101A800083270900D5EF79C43C486389F50817F727
:101A900001001307E7A363FCB7001443638D860CB2
:101AA00018434457B3B4950093C4140029A00443C9
:101AB000818C93B4140058546384E70A1C4C2CC8DE
:101AC00063C60700A947B385B7400CCC931727001E
:101AD000BA97584897F90100938989AE8A07CE973B
:101AE000631BF702130A44005285EFE07FA817F743
:101AF00001001307679C5C5418436376F70017F7DF
:101B00000100232BF79A5147B387E702D28533852B
:101B1000F900EFE07FA199C0EFE05F8F8327090014
:101B200081CB97F701009387A79A9C43FC439DEBD9
:101B3000F2406244D2444249B249224A056182805D
:101B400097F701009387C79898439C437C43850788
:101B50007CC31DF897F701009387879780432DB7C3
:101B60004CD4A9BF6244F240D2444249B249224A0D
:101B700005616F40406681443DBF25C1011126CA01
:101B800097F401009384C4949C4006CE22CC4AC8AA
:101B90004EC6638DA7027370043017F90100130954
:101BA00069918327090091C798409C407C43850731
:101BB0007CC3584997F70100938707B26302F70285
:101BC0008327090081C79C40FC43A5EBF240624497
:101BD000D2444249B249056182807370043001A049
:101BE0001C5517F701001307A7ACE38BE7FCE9FBD3
:101BF000930945002A844E85EFE09F9717F701006F
:101C00001307878B5C5418436376F70017F70100BE
:101C10002324F78A5147B387E70217F5010013051C
:101C2000259ACE853E95EFE03F909C405854DC5776
:101C3000E368F7F8EFE08FFD61B76244F240D24409
:101C40004249B24905616F40005915CD011122CCBE
:101C500026CA4AC82A8406CE4EC6EFE01F875848D7
:101C600097F70100938747A72A8981446300F70209
:101C70004A85EFE03F85F240624426854249D244DE
:101C8000B249056182807370043001A01C5417F5BD
:101C900001001305E5A1E38DA7FCF9FB97E701001F
:101CA0009387C77F9C43A9EB97F7010093874782EF
:101CB0009C43445493094400DC574E85B3B4F4006C
:101CC000EFE01F8B17E701001307077F5C541843F1
:101CD00093C414006376F70017E70100232EF77C06
:101CE0005147B387E70217F501001305658DCE85CF
:101CF0003E95EFE07F83ADBF93058401EFE0DF8287
:101D000085BF0111056506CE22CC26CA4AC84EC63B
:101D100052C456C25AC0EF200036630E051AAA8478
:101D200013050006EF2020352A84630A051C05668A
:101D30009305500A04D92685EF20205A0458856758
:101D4000F117BE94B7474C4593879744130A440054
:101D50005CD85285230C0402A30104042326040248
:101D600023280404232A0404EFE0AFFB13058401B5
:101D7000EFE02FFBA947232C0404F19800C81CCCEA
:101D800040D023220404232E0404014697150000AA
:101D90009385E5B12685EFE0EFF308C0737004305A
:101DA00017E90100130909718327090097E401006D
:101DB0009384047291C798409C407C4385077CC300
:101DC00017E701001307C76F1C43850797E601005B
:101DD00023A8F66E9C40C9C38327090097E9010038
:101DE0009389097E81EB9C40DC5789E797E70100E6
:101DF00023A0876E97E701009387C76A984397E609
:101E000001009386666B5C549442050717E6010057
:101E1000232AE66838C463F6F60017E70100232D8D
:101E2000F768139527003E950A05D2854E95EFE099
:101E3000AFEF8327090081C79C40FC43DDE7832780
:101E4000090091C39C40EF10704985476305F50C6C
:101E500059E17370043001A097E7010023AA876657
:101E60001843854797E9010093898975E314F7F8CA
:101E7000CE8A17FB0100130B2B815685D10AEFE0A8
:101E80000FE9E31C5BFF17E501001305E57FEFE0B9
:101E90000FE897FA0100938A6A805685EFE02FE7F2
:101EA00017F501001305C580EFE06FE617F5010097
:101EB00013054581EFE0AFE517F501001305C58176
:101EC000EFE0EFE497E7010023A2676197E70100E5
:101ED00023AC575F05B7F2406244D2444249B2494D
:101EE000224A924A024B05618280984094407C438A
:101EF000FD177CC3FC42A1F77360043089B76244CC
:101F0000F2404249B249224A924A024B2685D244C3
:101F100005616F20602873700430FD5717E70100DA
:101F20002320F758624497E7010023A5A758F24001
:101F3000D2444249B249224A924A024B97E70100F1
:101F400023AE075605616FE0CFB57370043097E795
:101F5000010023A107566FE00FC317E70100130725
:101F6000E7531C4385071CC382807370043097E7D6
:101F7000010093872754984305E317E701001307EF
:101F8000E75308439C4381CB97E70100938747546D
:101F90009843784301EF828017E701001307475306
:101FA00014431843F8420507F8C2C1BF984394434D
:101FB0007C43FD177CC3FC42F9FF736004308280D0
:101FC000411106C622C4EFE04FD097E70100938786
:101FD000E74E8043EFE00FCFB2402285224441011B
:101FE000828097E701009387A74D884382807971AB
:101FF00006D622D426D24AD04ECE52CC56CA5AC881
:102000005EC697E70100938767499C43B1EF17E7E6
:1020100001001307A74A1C43850797E6010023AF79
:10202000F648832A0700638F0A0697E70100938723
:1020300027479C43814463F1FA0897E9010093899B
:10204000295817EA0100130AAA4883270A0085467F
:10205000D85793172700BA978A07BE9983A7090014
:1020600063FFF600854421A897E701009387474462
:102070009C438144850717E70100232BF74297E72C
:1020800001009387A7429C4391C38544B2502254D8
:10209000268502599254F249624AD24A424BB24BC7
:1020A0004561828017E40100130444421C409C43B4
:1020B000DDC37370043001A017E401001304044170
:1020C00097E901009389C94F17EA0100130A4A40B2
:1020D00017EB0100130B4B3E1C409C43B5C31C4047
:1020E000DC4703A9C70083274900930B49005E859D
:1020F00063EEFA04EFE0CFC7832789021305890155
:1021000099C3EFE0EFC68327C90203270B00DE85E2
:10211000139527003E950A054E956376F70017E75D
:102120000100232BF738EFE02FC083270A00032795
:10213000C902DC57E362F7FA1C4085449C43C5F3AF
:10214000FD5717E70100232DF73401B717E701000A
:102150002328F734DDBD17E701001307E7361C40DD
:10216000184397E6010023A3E63617E70100232D65
:10217000F73497E70100938727339C43850717E7D8
:1021800001002323F7321C409C4399E7FD5717E7D2
:1021900001002327F73051BD1C40DC47DC47DC43FE
:1021A00017E70100232EF72E49B597E70100938723
:1021B000E72E984301E77370043001A0011106CEA9
:1021C00022CC26CA4AC84EC652C456C25AC07370E0
:1021D000043097E401009384E42D984061EB984328
:1021E0007D1797E6010023ABE62A9C43D9EB97E7DE
:1021F00001009387E72C9C43C9C797EA0100938AA3
:102200002A3C17EA0100130A2A2B17E901001309D7
:10221000292C854919A83385EA00EFE0EFB0832720
:1022200009005854DC576379F70483A70A0FC1CF1C
:1022300083A7CA0FC04713058401EFE06FB3130BE8
:1022400044005A85EFE0CFB25C5483260A00DA8559
:10225000139527003E950A052A875695E3FDF6FA61
:1022600017E70100232AF724EFE00FAC83270900CA
:102270005854DC57E36BF7FA97E7010023A837239C
:102280006DB701449C4081CB97E7010093874724B9
:102290009C43FC4395E72285F2406244D244424984
:1022A000B249224A924A024B0561828017E7010037
:1022B0001307072214431843F8420507F8C205B76D
:1022C000EF307071C9BF17E401001304641E1C4095
:1022D00095C31C40054999CF193B09C597E70100F3
:1022E00023A6271D1C40FD1717E701002322F71C1A
:1022F0001C40FDF397E701009387471B98438547F0
:10230000E311F7F8EFE08F900544ADBF11CD81E503
:102310007370043001A017E70100130727181C434E
:1023200099C77370043001A07370043001A041118B
:1023300022C406C614431841850617E60100232F60
:10234000D61497E601009386661794423304B700CB
:1023500000C163F7E602637FE40063FD860097E750
:1023600001009387E71688431105EFE06FA02285EF
:10237000EF3030601D3D01C9B240224441018280EE
:10238000E36FE4FCD9BF2244B24041016FE00F8803
:1023900011C917E70100130767101C4391C7737039
:1023A000043001A06FE08F86411106C622C4184395
:1023B000AA87050797E6010023A2E60E97E601002B
:1023C0009386061117E701001307470F1843884249
:1023D0003304F7001105EFE0AF992285EF30705913
:1023E000E93311E52244B24041016FE02F82B2404F
:1023F000224441018280411122C406C697E70100B0
:102400009387C7099C430144850717E701002327E9
:10241000F70897E701009387A70A9C4363E0F5124A
:1024200017EE0100130E8E2597E2010093828218A9
:1024300001440147854F1303500A21A0311E638DCB
:10244000C20B83278EFFBA86F5DB8327CEFFDC43E2
:10245000232EFEFE638AC70F03AFC700DC432A9713
:10246000814E232EFEFE6385C70783A8C70093878E
:102470004803232017015CC383A788042326F701A0
:102480001CC783A7C8021CCB83A70805232C070001
:102490005CCB03A808038347080063906704C287E6
:1024A000850783C60700B3850741E38B66FE8981F4
:1024B000C205C181231EB700850E130707026306FC
:1024C0001F038327CEFFDC43232EFEFEE39FC7F9C5
:1024D00083274E00232EFEFE49BF8145231EB700F1
:1024E000850E13070702E31E1FFD76941317540091
:1024F000311EBA86E397C2F597E70100938707FD7F
:1025000003AE070083270E00639D070E97E70100C7
:10251000938787FB03AE070083270E00639207189B
:1025200017EE0100130ECE0983274E109DE383277B
:102530008E116395072019C223200600BD31228524
:10254000B24022444101828083274E00232EFEFEAA
:1025500021B783278E1017EF0100130F2F17DC43CD
:1025600017E701002322F7166380E73383A2C70031
:10257000DC43AA96814E17E701002327F714914FF9
:102580001303500A6388E70783A8C70093874803AB
:1025900023A01601DCC283A7880423A6F6019CC6EB
:1025A00083A7C8029CCA83A7080523AC0600DCCA1F
:1025B00003A80803834708006391672AC287850739
:1025C00003C70700B3850741E30B67FE93D72500D8
:1025D000C207C183239EF600850E9386060263869A
:1025E000122983278E10DC4317E70100232EF70CF6
:1025F000E39CE7F983270E1117E701002326F70C68
:1026000061B783274E00130F8E00D4432322DE00D0
:102610006388E629B307E500D84283A2C600814E4D
:102620002322EE00894F1303500A6306EF06832826
:10263000C7001387480323A01701D8C303A7880442
:1026400023A6F70198C703A7C80298CB03A70805DC
:1026500023AC0700D8CB03A808030347080063187E
:10266000671C4287050783460700B3050741E38BD4
:1026700066FE13D7250042074183239EE700850E9F
:1026800093870702638D121B83264E00D8422322B4
:10269000EE00E31EEFF80327CE002322EE0041BF39
:1026A00083274E00130F8E00DC432322FE00638439
:1026B000E71F83A2C700DC43AA96814E2322FE00B7
:1026C000894F1303500A6306FF0683A8C700938748
:1026D000480323A01601DCC283A7880423A6F601C1
:1026E0009CC683A7C8029CCA83A7080523AC060022
:1026F000DCCA03A808038347080063966710C287F3
:10270000850703C70700B3850741E30B67FE93D72F
:102710002500C207C183239EF600850E938606021C
:10272000638B120F83274E00DC432322FE00E31E3F
:10273000FFF88327CE002322FE0041BF8327CE115E
:1027400097EE0100938ECEF9DC4317E701002327B3
:10275000F7F86384D71383AFC700DC433307D50092
:10276000014397E6010023ABF6F60D4F894293082B
:10277000500A6387D707C8479307450308C35CC35C
:102780003C452326E7011CC75C551CCB1C5599C34F
:10279000232657003C49232C07005CCB0328050364
:1027A0008347080063951705C287850783C607001E
:1027B000B3850741E38B16FF93D72500C207C1837A
:1027C000231EF700050313070702638AAF0283275E
:1027D000CE11DC4397E6010023A2F6F0E39DD7F982
:1027E00083274E1297E6010023AAF6EE69B78147C8
:1027F000231EF700050313070702E39AAFFC1A94A0
:10280000E31C06D225BB8147239EF600850E9386E6
:102810000602E39912F117EE0100130E6EDA832718
:102820004E10769493165400E38307D01DB30147EE
:10283000239EE700850E93870702E39712E597E74B
:102840000100938767C803AE07007694931654007F
:1028500083270E00E38607CCA1B58147239EF600AF
:10286000850E93860602E39E12D783278E117694F7
:1028700093165400E38107CCD1B583274E1217E796
:102880000100232DF7E4C1BD83270E1117E70100D6
:10289000232CF7E2E1B98327CE002322FE0011BDED
:1028A0008326CE002322DE00B5B3797126D24AD02A
:1028B0004ECE52CC56CA5AC85EC606D622D497E926
:1028C00001009389A9BD17E90100130969CF17EA2F
:1028D0000100130A2ABE97EA0100938A6ABF97EBA8
:1028E0000100938BEBBD97E401009384A4BD054BDD
:1028F00021A883A7090003244910850717E70100D1
:10290000232EF7B85D3011E89C40E5F783270900D6
:10291000E37CFBFEEFD09FAFC5BF7370043083270D
:102920000A00B9E383270911C04713054400EFD01B
:102930003FC483A70B00FD1717E701002322F7B858
:102940009C40FD1717E70100232EF7B683270A00E6
:1029500089C783A70A00FC4385E30858EF10D0031A
:102960002285EF1070034DB703A70A0083A70A0062
:102970007C4385077CC37DB703A70A0083A60A00B2
:102980007C43FD177CC3FC42E9FB73600430F1B764
:1029900097E70100938787B09C43DDE3411106C6AA
:1029A00097E7010023A407B017E70100130747B218
:1029B0001C43B7A6A5A59386565A9C5B8C43639B84
:1029C000D500D0436318B60094476395C600DC4732
:1029D0006388D70008430C4393854503EF20C073F9
:1029E00097E60100938646AD904217E70100130772
:1029F00027BD11A89C42B9CB9C42FD1717E60100E8
:102A0000232CF6AA904293172600B2978A07BA970A
:102A10009C43EDD3904293172600B2978A07B305E3
:102A2000F700D441A107BA97D442D4C16383F60218
:102A3000DC46B24017E70100232CF7A84101828051
:102A4000854717E701002323F7A6828073700430BF
:102A500001A0D1473306F602D442329754C3C9BF0E
:102A600001114AC806CE22CC26CA4EC62A897370E6
:102A7000043097E401009384E4A39C4017E4010030
:102A8000130404A5D9E7631409000329040093097A
:102A900049004E85EFD0DFAD8327890289C7130532
:102AA0008901EFD0FFACCE8517E501001305C5C243
:102AB000EFD09FA79C4081C71C40FC43ADE31C4066
:102AC000638B27079C409DCF737004309C40C1EB03
:102AD00097E701009387879F9843184325EBFD579D
:102AE00017E70100232EF79A9C4089CF1C40FC4336
:102AF00091CB184014407C43FD177CC3FC4299E302
:102B000073600430F2406244D2444249B2490561E4
:102B1000828018401C407C4385077CC3ADB71840B9
:102B200014407C43FD177CC3FC42D1FB736004302E
:102B30001C40E39927F99C40A1C397E701009387C4
:102B4000E7959C43ADCB7370043001A09C43DC47F8
:102B5000DC47DC4317E701002324F79471B71840E2
:102B60001C407C4385077CC397E701009387079649
:102B7000984318432DD7D9BF97E70100938747940F
:102B800017E701001307C7A39C4303278711631DA1
:102B9000F700F240624497E7010023AB0792D2446A
:102BA0004249B249056182806244F240D2444249BE
:102BB000B2490561F1BB6244F240D2444249B24994
:102BC00005616FD0BF843DC9411126C297E4010061
:102BD000938404904AC02E898C4006C622C4E10525
:102BE000EFD01F9688401105EFD09F98FD57630ADC
:102BF000F90497E701009387678C804398409C43D2
:102C00004A9440C3636CF40497E701009387078CF0
:102C100088438C409105EFD0BF9297E701009387DE
:102C200027889C436376F40097E7010023AA8786F0
:102C3000B2402244924402494101828073700430C0
:102C400001A08C402244B2409244024917E50100A1
:102C5000130585A8910541016FD01F8D97E70100ED
:102C600093878786884322448C40B240924402492D
:102C7000910541016FD0DF8C11C997E7010093875F
:102C8000E7819C4399E77370043001A073700430AE
:102C900001A0411126C297E4010093846483984007
:102CA000AE878C40B7060080D58F06C622C41CCFE5
:102CB000E1053284EFD05F8788401105EFD05F8B4C
:102CC000FD57630EF40097D701009387277F884351
:102CD000B24092442295224441016F3080498C4099
:102CE0002244B240924417E501001305E59E910588
:102CF00041016FD07F8325CD411126C297D40100B9
:102D00009384047D4AC02E898C4006C622C4E10506
:102D10003284EFD07F8188401105EFD07F858547D1
:102D2000630AF40497D7010093874779804398405A
:102D30009C434A9440C3636CF40497D70100938783
:102D4000E77888438C409105EFD08FFF97D701003B
:102D5000938707759C436376F40097D7010023A1FE
:102D60008774B240224492440249410182807370C8
:102D7000043001A08C402244B2409244024917E53D
:102D8000010013056595910541016FD0EFF997D7C3
:102D9000010093876773884322448C40B240924479
:102DA0000249910541016FD0AFF9411106C622C415
:102DB00026C25C45C04735CC930484012685EFD0FC
:102DC0002FFB97D701009387676D9C43B5E793046A
:102DD00044002685EFD0CFF997D701009387C76DC0
:102DE00058549C4363F6E70097D7010023A6E76C8D
:102DF00093172700BA978A0717D501001305457C5A
:102E0000A6853E95EFD04FF297D701009387476C88
:102E10009C4358540145DC5763F8E700854717D7B2
:102E200001002325F7680545B24022449244410140
:102E300082807370043001A0A68517E50100130598
:102E40002587EFD06FEEC9B797D701009387076545
:102E50009C4381E77370043001A0411106C622C46F
:102E600026C2B70700804045CD8F1CC12DC4EFD0CE
:102E70002FF0930444002685EFD08FEF97D7010001
:102E80009387876358549C4363F6E70097D7010004
:102E900023A4E76293172700BA978A0717D5010082
:102EA000130505723E95A685EFD00FE897D7010070
:102EB000938707629C4358540145DC5763F8E70049
:102EC000854717D701002323F75E0545B24022440A
:102ED0009244410182807370043001A011CD97D7D4
:102EE00001009387675C984397D701009387075D3C
:102EF0009C4318C15CC182807370043001A055C12D
:102F0000D1CD411106C622C42A877370043097D8E8
:102F100001009388285A83A7080091CB97D7010016
:102F20009387075B94439C43FC428507FCC217D3FD
:102F300001001303A3589C4103260300FD560144DE
:102F4000638FD70217DE0100130E0E5603250E0005
:102F50000328070054436305A80005446371D602A3
:102F60003308D6400544637CF80003250E00918F9A
:102F700003260300B6979CC108C350C3014483A72E
:102F8000080081CB97D70100938787549C43FC436B
:102F900081EF2285B2402244410182807370043067
:102FA00001A07370043001A0EF30E022DDB7854747
:102FB00017D70100232CF74E828019C16845828003
:102FC0000145828011C16CC5828097D7010093872B
:102FD00027508843828097D701009387A74D9C4351
:102FE000054589CB97D701009387474B8843133515
:102FF00015000605828031CD011126CA97D4010043
:103000009384044D9C4006CE22CC4AC84EC65855E7
:10301000DC576379F7021C4D63C707009C40D45707
:10302000A947958F1CCD93172700BA97584917D9F0
:1030300001001309E9588A07CA97630DF7009C40FD
:10304000DC575CD5F2406244D2444249B249056142
:1030500082808280930945002A844E85EFD04FD12B
:103060009C4017D70100130727451843DC575CD451
:103070006376F70017D701002320F7441395270044
:103080003E9562440A05F240D244CE854A95B24943
:10309000424905616FD04FC919CD411106C622C4FE
:1030A00026C297D701009387A74280436307A400F5
:1030B0007370043001A0014582807C4881E7737001
:1030C000043001A054543848FD177CC86383E600DF
:1030D00099C70145B2402244924441018280930441
:1030E00044002685EFD0CFC83C4817D7010013070E
:1030F000A73C144329471D8F5CD418CC63F6F60017
:1031000017D70100232AF73A5147B387E70217D5AB
:1031100001001305E54AA6853E95EFD0EFC00545B1
:1031200055BF7370043097D701009387A7389C432D
:1031300091CB97D701009387A73998439C437C4351
:1031400085077CC3828097D701009387A7369C436D
:103150008DC397D701009387A7379843784311CB46
:10316000984394437C43FD177CC3FC4299E373600E
:103170000430828097D7010093878735904394432A
:103180009843A947D456084E958F1CCF828097D775
:1031900001009387E733984309C79443F84A05072A
:1031A000F8CA8843828079714AD006D622D426D2C2
:1031B0004ECE2A897370043097D401009384842FF3
:1031C0009C4017D401001304A430BDE31C40BC4F45
:1031D00089E71C400547F8CFD1E19C4081C71C40DE
:1031E000FC43F1EB737004309C408DEF1C40A84F02
:1031F00011C5630409021C4023AC07041C4023AE24
:1032000007049C4081C71C40FC438DEBB250225404
:1032100092540259F2494561828018403C4FFD1793
:103220003CCFE9BF18401C407C4385077CC37DBF71
:1032300018401C407C4385077CC349BF184014409C
:103240007C43FD177CC3FC42F1F373600430B25041
:10325000225492540259F2494561828008402EC698
:103260001105EFD0EFB0B245FD576380F50697D753
:1032700001009387A72483A9070018409C43AE99B7
:103280002322370163ECF90497D7010093870724C1
:1032900088430C409105EFD0AFAA97D701009387E0
:1032A00027209C4363F6F90097D7010023AA371F14
:1032B000EFD0CF951DB7184014407C43FD177CC359
:1032C000FC428DF37360043031BF0C4017D5010010
:1032D000130585409105EFD02FA5D9BF97D70100E1
:1032E0009387871E88430C409105EFD06FA5C9B71F
:1032F00079714AD04ECE06D622D426D252CC2E890F
:10330000B2897370043097D401009384A41A9C404E
:1033100017D401001304C41BF9EF18408947784FF4
:10332000630CF7001C401345F5FFB84F798DA8CF0B
:103330001C400547F8CFADE69C4081C71C40FC43CC
:10334000F5E3737004309C40B1E7638609001C40CC
:10335000BC4F23A0F900184085470145784F630B07
:10336000F7001C401349F9FF0545B84F3379E900D0
:1033700023AC27051C4023AE07049C4081C71C409A
:10338000FC43C1E3B250225492540259F249624ABA
:103390004561828018401C407C4385077CC375B71B
:1033A000084036C61105EFD0AF9CB246FD57638585
:1033B000F60897D701009387671003AA0700184003
:1033C0009C43369A232247016363FA0897D701008A
:1033D0009387C70F88430C409105EFD06F9697D71E
:1033E00001009387E70B9C436370FA0697D70100AF
:1033F00023A8470B91A818401C407C4385077CC339
:1034000029BF184014407C43FD177CC3FC42BDFB20
:1034100073600430B250225492540259F249624A05
:1034200045618280184014407C43FD177CC3FC42F8
:1034300089FB7360043031B70C4017D501001305C8
:10344000A5299105EFD04F8EEFC05FFCF5B597D75A
:1034500001009387670788430C409105EFD04F8E9A
:10346000E5B751C1411106C622C426C24AC07370D5
:10347000043097D401009384E4039C40B9EB99C2D3
:103480003C4D9CC2B2878946704D74CD2E872A84EC
:103490006386D70663FCF6048D456387B7009145C4
:1034A0006395B7006300D60C38CC8547630FF604EC
:1034B00005449C4081CB97D70100938767019C43CB
:1034C000FC43A9E32285B2402244924402494101CF
:1034D000828097D701009387A7FF98439C437C4342
:1034E00085077CC369BF7370043001A08546E39EE5
:1034F000D7FA3C4D33E7B70038CD45BF3C4D850783
:103500003CCD65B7EF20304D75BF130944004A85A7
:10351000EFD00F8617D70100130707FA5C54184342
:103520006376F70017D701002328F7F85147B387D0
:10353000E70217D501001305A508CA853E95EFC01F
:10354000BFFE1C5481C77370043001A097D70100DF
:10355000938707F89C435854DC57E3FBE7F4EFC02C
:10356000FFEAB9B70144B1B739CD011122CC26CA5F
:103570004AC84EC652C456C206CEBA89368AB284EA
:103580002E892A84EFC07FF4AA8A63050A003C4C86
:103590002320FA00784C89477CCC6389F40263F4D9
:1035A000970C8D466387D40091466396D400630AD6
:1035B000F70A232C24058547631EF7061C5499CB74
:1035C0007370043001A07370043001A03C4C850777
:1035D0003CCCD5B797D70100938747EC9C43ADEB24
:1035E000930444002685EFC0BFF817D701001307E6
:1035F000A7EC5C5418436376F70017D70100232D1E
:10360000F7EA5147B387E70217D50100130545FBD9
:10361000A6853E95EFC05FF197D70100938747EBF2
:103620009C435854DC5763F7E700638509008547DE
:1036300023A0F90005445685EFC0DFE82285F2405B
:103640006244D2444249B249224A924A0561828088
:103650009305840117D5010013058505EFC0DFEC44
:1036600065BF0144C9BF8547E397F4F43C4C33E997
:103670002701232C240581B74DC1011122CC26CA74
:103680002A844AC806CE4EC6AE84EFC01FE48947DE
:10369000744C7CCC3C4C05472A8985073CCC63950F
:1036A000E6061C5481C77370043001A097D701004F
:1036B0009387C7DE9C43ADE7930944004E85EFC076
:1036C0003FEB17D70100130727DF5C5418436376DD
:1036D000F70017D701002321F7DE5147B387E70230
:1036E00017D501001305C5EDCE853E95EFC0DFE38C
:1036F00097D701009387C7DD9C435854DC5763F587
:10370000E70099C085479CC06244F240D244B24968
:103710004A85424905616FC0FFDA7370043001A029
:103720009305840117D50100130585F8EFC0DFDF8D
:10373000C1B7AA8729C57370043017D701001307D2
:1037400067D714439DE2F04F894601456315D600C3
:1037500023AE070405451C4381CB97D7010093870F
:1037600027D79843784315E3828097D60100938644
:1037700026D6904294427442850674C2E9B797D720
:1037800001009387E7D49C437DB7984394437C43DF
:10379000FD177CC3FC42E9FB7360043082805D71DD
:1037A000A6C2CAC052DC56DA5AD85ED686C6A2C4B1
:1037B0004EDE62D466D26AD017D90100130949D20D
:1037C00017DB0100130B0BD197D401009384C4D0F5
:1037D00097DA0100938A8AD0054AA54B832709000E
:1037E000984363010712DC4783A90700EFE0EFF677
:1037F000EFE0AFF783270B002A8C6362F50A97D7B7
:10380000010023A9A7CC01466370351B8840B3850E
:103810008941EFD0FFBDEFE05F9963010512884059
:10382000814601462C00EFD00FEC4DD9A247E3C8EA
:1038300007FEC24983A7490189C713854900EFC024
:103840003FD3EFE08FF283270B002A8C636DF508DE
:10385000A24717D70100232F87C7E3E2FBFCB3176A
:10386000FA0013F70721631A071613F7770C63188A
:10387000071E93F70702C5D74E85EF00F01145B735
:10388000DC47C04783AC0700930944004E85EFC076
:103890003FCE5C50228582975C4C6384470B832724
:1038A0000900984371FF03A70A0097D6010023A3DC
:1038B00086C397D6010023A3F6C297D7010023A1A0
:1038C000E7C2EFE09F8EA1BFDC47C04703AD070012
:1038D000930C44006685EFC0BFC95C502285829777
:1038E0005C4C6386470983270900984371FF03A74F
:1038F0000A0097D6010023A3F6BE97D7010023A1A3
:10390000E7BEB9B7EFE06FE5EFE02FE683270B00E6
:103910002A8CE366F5F883A70A0088408149904322
:10392000B385894117D70100232687BB13361600BC
:10393000EFD01FACEFE07F87E31305EEEFC01FADC4
:10394000F9BD1C4CCE85E69763E9FC049C4089CF09
:1039500002CA66CC22CEEFF00FE8884081460146CD
:103960004C08EFC05FE205FD7370043001A01C4CF1
:10397000E685EA97636CFD049C4089CF02CA6ACC55
:1039800022CEEFF04FE58840814601464C08EFC05B
:103990009FDF31F97370043001A0032509005CC07A
:1039A00000C8EFC0FFB9E5BDEFE03F808327090005
:1039B000DC47C047930C44006685EFC07FBB5C4C7E
:1039C000638F47035C502285829791BD03250900D0
:1039D0005CC000C8EFC0DFB639B7B24723ACF9000E
:1039E000A5CFE29723A2F90023A8390193854900C6
:1039F000636FFC0403A50A00EFC09FB40DB51C4C17
:103A000000C83387F90058C0636DEC02330C3C41A9
:103A10006363FC029C4089CF02CA4ECC22CEEFF0F9
:103A20008FDB8840814601464C08EFC0DFD559F94D
:103A30007370043001A003A50A00E685EFC05FB0F3
:103A400051B703250900E685EFC09FAFA5BF032549
:103A50000900EFC0FFAEE1B37370043001A0B247BC
:103A600083A6890123A839013387D70023A2E9005F
:103A70006364EC04B307FC4063EBD70483A74902FB
:103A80004E85829783A7C901E39B47D983A6890105
:103A9000B2479840B69711CF02CA3ECC4ECEEFF057
:103AA0008FD38840814601464C08EFC0DFCDE31834
:103AB00005D67370043001A06374FC00E370F7FC5A
:103AC0000325090093854900EFC09FA789BB03A583
:103AD0000A0093854900EFC0BFA691B3411122C4EB
:103AE00006C626C24AC017D401001304E49EEFF0B4
:103AF0004FE31C4095CBEFF00FE51C409DC3814880
:103B000001488147094781461306004097D50100C7
:103B10009385C58A170500001305A5C8EFD07F9AC5
:103B200039E97370043001A017D90100130909BCE9
:103B30004A85EFC0DF9D97D40100938464BC26853D
:103B4000EFC0FF9C0146B145114597D7010023A95D
:103B5000279997D7010023A39798EFC03FB617D7AF
:103B60000100232BA79611CD97D50100938585845D
:103B7000EFD0CFFC49B7B240224492440249410100
:103B800082807370043001A0A5C9797156CAAA8ACF
:103B90001305C00222D426D24AD04ECE52CC06D62D
:103BA0005AC85EC63A89B689328AAE84E9212A8427
:103BB00005C9EFF00FD797D701009387E7919C4392
:103BC0009DCFEFF04FD8130544002320540104CCBF
:103BD000232E44012320340323222403EFC07F94A7
:103BE0002285B250225492540259F249624AD24A72
:103BF000424BB24B456182807370043001A097DB69
:103C00000100938BABAE5E85EFC07F9017DB0100A8
:103C1000130B0BAF5A85EFC09F8F0146B14511457D
:103C200097D7010023AE778B97D7010023A8678B26
:103C3000EFC0DFA817D701002320A78A01C997C5C5
:103C4000010093852577EFD06FEFA5BF7370043027
:103C500001A039C5011122CC06CE26CA17D4010015
:103C600013048487832804002A8801456385080299
:103C7000BA842EC2368732C442C6954663C5B602A0
:103C8000EFF06FB58947630BF502084081460146A6
:103C90004C00EFC05FAFF2406244D24405618280C5
:103CA0007370043001A04C0081463A864685EFD0FF
:103CB0000F88F2406244D244056182800840814608
:103CC00026864C00EFC03FACF9B719C1084182808D
:103CD0007370043001A001E57370043001A041113C
:103CE00006C622C42A84EFF0CFC348483334A0006C
:103CF000EFF06FC52285B24022444101828001E588
:103D00007370043001A0411122C42A8406C6EFF06A
:103D10004FC10050EFF02FC3B24022852244410131
:103D2000828001E57370043001A0411122C426C2D3
:103D30002E84AA8406C6EFF0CFBE80D02244B240C3
:103D4000924441016FF02FC04111714522C406C653
:103D50001D262A8411C5232005001105EFC02FFB65
:103D60002285B24022444101828001CDB70700FF85
:103D7000ED8F81C77370043001A099E57370043032
:103D800001A07370043001A0011122CC4AC84EC6B4
:103D900052C456C206CE26CABA893689B28A2E8441
:103DA0002A8AEFF04FA311E5638509007370043090
:103DB00001A0EFE08F9A83240A00B3779400631682
:103DC000090295C763870A009347F4FFE58F232014
:103DD000FA00EFE08FBDF240624426854249D244AA
:103DE000B249224A924A05618280E30DF4FCE382E3
:103DF00009FEB3355001E20563050900B707000469
:103E0000DD8D4E86C18D13054A00EFE0FFE6EFE041
:103E1000CFB919E1EFC08FDFEFF0CFB59317650091
:103E2000AA8963D80700B7040001FD14B3F4990010
:103E30005DB7EFF00FAF83290A00B3773401631E3B
:103E4000090089CB63880A009347F4FFB3F7370171
:103E50002320FA00EFF02FAFF9B7E31DF4FEDDB732
:103E600001C9B70700FFED8F99C77370043001A037
:103E70007370043001A0411122C42A8406C626C2F0
:103E80004AC02E89EFF0EFA904409345F9FFB3F73C
:103E900095001CC0EFF02FABB240224426850249AA
:103EA000924441018280411122C42A8406C6EFC097
:103EB000CFE10040EFC00FE1B24022852244410132
:103EC000828009C9370700FFB3F7E50099C773700F
:103ED000043001A07370043001A06F208031B70757
:103EE00000FFF18F81C77370043001A001E6737089
:103EF000043001A0011122CC4AC84EC652C406CEDD
:103F000026CA3689AE892A8A3284EFF0CF8C21E125
:103F1000630509007370043001A0EFE00F8483246F
:103F20000A00CE855285B3E49900613FB3779400CF
:103F30006307F40683240A00EFE02FA7F2406244EF
:103F400026854249D244B249224A05618280EFE087
:103F5000CF8083240A00CE855285B3E4340195379F
:103F6000B3F78400638D8702E30609FCB7050005FB
:103F70004A86C18D13054A00EFE01FD0EFE0EFA2A3
:103F800019E1EFC0AFC8EFF0EF9E93176500AA8468
:103F900063DF0700B7070001FD17FD8C45B78327D6
:103FA0000A001344F4FFE18F2320FA0071B7EFF009
:103FB0004F9783240A00B377940063978700934751
:103FC000F4FFE58F2320FA00EFF0EF97E1B74111FE
:103FD00022C406C62A8426C2EFD03FF85C4085C3BF
:103FE00008489304C4006316950015A008486300B0
:103FF0009502B7050002EFE03FE55C40E5FB228556
:10400000612A2244B240924441016FE00F9A7370DA
:10401000043001A009C9370700FFB3F7E50099C7CD
:104020007370043001A07370043001A06F20601C15
:1040300001C9B70700FFED8F99C77370043001A065
:104040007370043001A0411122C426C206C62A841E
:10405000AE84EFF00F8D184093C7F4FFF98F1CC0AA
:104060002244B240924441016FF0EF8D19C1084DD6
:10407000828001458280411122C406C62A84EFD085
:10408000DFED97C701009387E7459C43A1EBE56708
:1040900017C7010013074768F11797C6010023A946
:1040A000E64417C701002323F74417C7010023275D
:1040B000F76697C701009387274317C70100232D91
:1040C000F764854717C701002326074217C7010079
:1040D000232C074017C701002326F74019E8EFE01B
:1040E000CF8CEF10E00201442285B240224441010E
:1040F00082801305840093773500C1EFE5671307CD
:10410000F5FFE917E3EDE7FC97C601009386463E0D
:104110009C4229A0984311C7BE86BA87D843E36B57
:10412000A7FE17C701001307273CE38AE7FA984365
:1041300041461384870098C2D843B306A7406378EA
:10414000D6023388A7002322D800C8C3832548009D
:1041500097C601009386C63911A0BA86984250438B
:10416000E36DB6FE2320E80023A00601D84397C7DD
:1041700001009387273B9C43998F17C70100232396
:10418000F73AEFE08F8231DC2285B24022444101D0
:104190008280719911059DB729C9411122C406C6B3
:1041A0002A84EFD09FDB930584FF0326C4FF17C743
:1041B00001001307E73311A03E871C43D443E3ED0E
:1041C000C6FE232CF4FE0CC397C7010093878735E6
:1041D00098438327C4FF2244B240BA9717C701000F
:1041E0002322F73441016FD05FFC828097C7010022
:1041F000938747338843828082803367B5000D8B75
:10420000AA871DE79308D6FFAA982A87AE8663710E
:10421000150303A8060011079106232E07FFE36A82
:1042200017FF9347F5FFC697F19B9107BE95AA9795
:104230002A9663F3C70A9386450013884700B3B6EE
:10424000D70033B8050133E7F50093C616001348CD
:1042500018000D8BB3E6060113371700758F330E68
:10426000F6409386170029CF1337AE0031EB135376
:104270002E002E88BE8601478328080005071108F6
:1042800023A016019106E36967FE1377CEFFBA9566
:10429000BA976302EE0483C60500138717002380D4
:1042A000D700637AC70283C6150013872700A3804F
:1042B000D7006372C70203C725002381E70082800D
:1042C000B307F640AE97850503C7F5FF8506238F34
:1042D000E6FEE39AF5FE82808280B367C5008D8B8F
:1042E000B308C500E9C36371150FB307A0408D8BF8
:1042F00013873700954693F5F50F130815003383A0
:10430000A8407D166373D70015476363E60CD5CFCD
:104310002300B5000547638DE700A300B5000D47F6
:10432000130825006396E700130835002301B50044
:10433000139685004D8E13970501518F3303F3407B
:1043400093968501D98E13562300AA97014794C3EB
:1043500005079107E36DC7FE1377C3FFB307E800B6
:104360006307E3062380B70013871700637C1703F6
:10437000A380B70013872700637617032381B70054
:104380001387370063701703A381B70013874700B3
:10439000637A17012382B7001387570063741701EC
:1043A000A382B700828093F5F50F13978500D98D0E
:1043B000139705014D8FE37715FFAA87910723AE69
:1043C000E7FEE3ED17FF828082802A8895B782801E
:1043D000AA8749BF834705002A8799C705058347F0
:1043E0000500EDFF198D8280014582800505834718
:1043F000F5FF850503C7F5FF91C7E389E7FE338520
:10440000E74082808147E5BFAA87850503C7F5FF9E
:104410008507A38FE7FE75FB82808346050093071F
:1044200000026397F600050583460500E38DF6FE5E
:10443000938756FD93F7D70F85C7AA87814585CE09
:1044400001458507138606FD1317250083C607005F
:104450003A9506053295F5F699C13305A04082805C
:10446000938536FD8346150093B515009307150017
:10447000E1FA0145D5B7014582809C412380A70020
:104480009C4185079CC1828097C601009386C60621
:104490009C42175703001307E72A13861700BA97A1
:1044A0002380A70097C5010023A8C504A947630876
:1044B000F500930700046305F6000145828075DE70
:1044C000370610F005078347F7FF2320F6F09C42DC
:1044D000FD1797C5010023A1F502EDF70145828084
:1044E0004D712322911423202115232A51132324B3
:1044F00081132326111423248114232E3113232CFA
:10450000411323286113232671132322911323209F
:10451000A113232EB111AA842E8932C6130C500286
:10452000A54A8347090063808703B9CB804011A067
:10453000A1CB2300F40080400509050480C0834717
:104540000900E39787FF0346190093081900C68600
:10455000130D0002FD597D5A0148130550059307BC
:10456000D6FD93F7F70F138916006363F52A17C773
:104570000100130727A98A07BA979C43BA97828735
:104580008320C114032481148324411403290114BA
:104590008329C113032A8113832A4113032B011397
:1045A000832BC112032C8112832C4112032D011283
:1045B000832DC11171618280A14C02C4854763D5EE
:1045C0000715B2478040938B770093F68BFF03ABC0
:1045D000060083A94600938786003EC6668681460C
:1045E0005A85CE85EF10B0032AC8814763853723EB
:1045F000930D4101854B668681465A85CE85EF1025
:10460000204C814666862A8BAE89EF105001A24766
:1046100023A0AD0093861B00910D63843701B68BF8
:10462000D9BFE37E9BFF63DD4601A2872380A701FC
:1046300080407D1A930714009CC03E84E3C846FF67
:1046400093962B001C08BE9631A89387770523000C
:10465000F4008040FD1B93871B00050480C0F11609
:10466000E351F0EC9C42E3E2FAFE93870703C5B7FF
:104670009C409306000332472380D7009C4093065A
:104680004700C14C1386170090C013068007A38013
:10469000C700804002C4BA87050480C003AB07008E
:1046A000814936C625BFB24783AC0700938B4700CC
:1046B00063840C1C635F40199307D0026319FD16D5
:1046C00083C70C0085C363DC09189440850C7D1AF0
:1046D0002380F6008040050480C083C70C00E5F706
:1046E000635D40018040930700022300F400804096
:1046F0007D1A050480C0E31A0AFE5EC61DB502C419
:104700008547A94CE3CF07EBB2478040938647002B
:1047100071B703C61600CA8699B59C40930650022D
:104720002380D7008040050480C0E5BBC14C02C493
:1047300071B5B24703C61600CA8683A90700910760
:104740003EC6E35E0AE04E8AFD5911BD03C616005F
:10475000130DD002CA8621B59347FAFFFD8703C621
:104760001600337AFA00CA86DDBB03C61600130DA5
:104770000003CA86EDB383C51600930906FDCA86F9
:10478000938705FD2E86E3EEFAFA93972900BE99EA
:1047900085068609AE9983C50600938909FD93872E
:1047A00005FD2E86E3F3FAFE69BF32479C401443B1
:1047B00011073AC62380D7008040050480C095B316
:1047C000854763D3070BB24793867700E19A9387B7
:1047D00086003EC683A946009C4263DC090A9440D9
:1047E0001306D002B307F0402380C6008040B336E2
:1047F000F000B3093041050480C03E8BB389D94035
:10480000A94C02C4E1BB03C616000508CA8681BBD9
:104810009C40468921B7E37D9BDD8547814B8546DA
:10482000E3C547E131BD97CC0100938CACB9CE858F
:104830006685EF00D06E330AAA40635C4001804079
:104840002300A40180407D1A050480C0E31A0AFEFB
:10485000014A83C70C00E38207EAE3C809E6FD19B1
:104860007D57E394E9E6ADBDB247938647009C438C
:1048700036C693D9F74195B7635640019307D002E6
:10488000E313FDFA97CC0100938CCCB3930780021D
:104890001DBD3E8BA94C02C4804089B34D71232EAF
:1048A0003113B70900409387F9FF23248114232291
:1048B0009114232C4113232A51132326111423204E
:1048C0002115232861132326711323248113232206
:1048D00091132320A113232EB1112A8A2EC417C4A9
:1048E0000100130464C1975A0300938AAAE597C490
:1048F00001009384A4863EC69305500229451308FF
:104900000004B70610F083470A006386B704C1C7E6
:104910001840050A13061700569797C8010023ADE3
:10492000C8BC2300F7006382A706E31E06FD1757E5
:104930000300130727E105078347F7FF23A0F6F0DD
:104940001C40FD1717C601002328F6BAEDF7834770
:104950000A00E39EB7FA83461A0013051A002A8755
:10496000930B00027D5B7D5C014893055005A548D3
:104970009387D6FD93F7F70F130A170063E7F53413
:104980008A07A6979C43A6978287175703001307A9
:1049900067DB55F28DBF8320C11403248114832467
:1049A0004114032901148329C113032A8113832A83
:1049B0004113032B0113832BC112032C8112832C6F
:1049C0004112032D0112832DC11171618280A14C0E
:1049D000014D854763DB0719A2479D07E19B83AD26
:1049E000070003AB4700138787003AC466868146F9
:1049F0006E85DA85EF10A0422AC863066D3513096B
:104A000041018549668681466E85DA85EF10400B47
:104A100066868146AA8D2E8BEF1060402320A90068
:104A200085091109E3106DFFE3FE9DFD13060004E7
:104A3000B70610F063D189031C4013871700D6977F
:104A400097C5010023AAE5AA23807701630CC70458
:104A50007D1CE3C389FFB2476800A548B386F9000F
:104A60008A061C08BE96294813030004370610F076
:104A7000E384A6E89C429305000363F4F8009305E1
:104A800070051840AE9793051700569717CE010092
:104A90002324BEA62300F7006380072B638C6526C2
:104AA000F116F9B7175703001307C7C9050783475E
:104AB000F7FF23A0F6F01C40FD1797C5010023ADBA
:104AC000F5A2EDF77D1C71B71C4013060004138797
:104AD000170097C5010023A1E5A2B386FA0093054C
:104AE00000032380B6006300C73E890797C6010014
:104AF00023A4F6A05697930680072300D7001757E4
:104B00000300130727C4B70610F0639EC70005070C
:104B10008347F7FF23A0F6F01C40FD1717C60100DE
:104B2000232CF69CEDF7A247C14C014D910722477B
:104B3000014B832D07003EC455BDA24783AC07003F
:104B400013894700638F0C3A635480219307D00286
:104B5000639EFB2E03C70C00BA856310072025ACAB
:104B60008547A94C014DE3C907E7A2479107C1B7A3
:104B7000A24783461700528703AB070091073EC444
:104B8000E3580CDE5A8C7D5BE5B383461700930B2C
:104B9000D0025287F1BB9347FCFFFD878346170085
:104BA000337CFC005287E9B383461700930B000364
:104BB00052877DBB03461700138B06FD5287930770
:104BC00006FDB286E3EEF8FA93172B00DA97050795
:104BD0008607B29703460700138B07FD930706FD70
:104BE000B286E3F3F8FE69BFA2451C40294698410E
:104BF00093861700D69717C50100232FD58E2380E3
:104C0000E700138945006301C72A930700046387FF
:104C1000F6204AC4D5B1854763DF0729A247138729
:104C20007700619B930787003EC4032B47001C431A
:104C3000635B0B301840130600049306170097C5FA
:104C4000010023ABD58A56979305D0022300B70005
:104C50006388C62CB307F0403337F000330B604154
:104C6000BE8D330BEB40A94C014D49B38346170071
:104C700005085287F5B9834617005287D5B91C40FD
:104C8000930600041387170017C601002326E68643
:104C9000D697130650022380C700E31FD7C41757C7
:104CA0000300130727AAB70610F005078347F7FF8D
:104CB00023A0F6F01C40FD1717C60100232EF68234
:104CC000EDF71DB9C14C014D29B31C4093060004FA
:104CD0002A8A1387170017C60100232FE680D6976C
:104CE000130650022380C700E318D7C017570300EC
:104CF000130747A5B70610F005078347F7FF23A062
:104D0000F6F01C40FD1717B601002327F67EEDF7DD
:104D10002A8ADDB6175703001307C7A20507834782
:104D2000F7FF2320F6F01C40FD1797B5010023A5DF
:104D3000F57CEDF7F1162DBB17570300130787A07D
:104D4000F1FDF11635B3E3FC9DCB8549C5B1014CAE
:104D500003C70C00BA85E30E07EAFD58294513087E
:104D60000004B70610F063570B0A1C4013861700A7
:104D7000D69717B301002321C3782380E70063840B
:104D8000A50663040609850C03C70C007D1CBA85C3
:104D900079FBE35080E91C409305000213060004F0
:104DA000B70610F021A07D1CE3050CE61387170061
:104DB000D6972380B70017B50100232FE572BA8775
:104DC000E313C7FE175703001307C7970507834769
:104DD000F7FF23A0F6F01C40FD1717B50100232DA7
:104DE000F570EDF7C9B7175703001307A79541DE14
:104DF00005078347F7FF23A0F6F01C40FD1717B601
:104E00000100232BF66EEDF7BDBF17570300130704
:104E10006793F9BF7D1BE31A1BF5A5BF1757030066
:104E200013074792B70610F005078347F7FF23A043
:104E3000F6F01C40FD1717B60100232FF66AEDF7B8
:104E40004AC45DBC97BC0100938CCC57DA8566855B
:104E5000EF00F00C330CAC40E35C80EF1C40130619
:104E60000004B70610F021A07D1CE3020CEE1387AE
:104E70001700D6972380770197B5010023AEE5662A
:104E8000BA87E313C7FE175703001307A78B05075D
:104E90008347F7FF23A0F6F01C40FD1797B50100EC
:104EA00023ACF564EDF7C9B71757030013078789DB
:104EB000B5FA4AC491B4A247138747009C433AC449
:104EC00013DBF741B5B3175703001307A787B706DE
:104ED00010F005078347F7FF23A0F6F01C40FD17ED
:104EE00017B60100232AF660EDF7854717B70100D2
:104EF0002324F76093078007175703002304F784E0
:104F00001DB1635680019307D002E39DFBF297BC6D
:104F10000100938C2C4B130780029305800235BD52
:104F20009756030093860682370610F0850603C75E
:104F3000F6FF2320E6F018407D1797B5010023AD5A
:104F4000E55A6DF701BBBE8DA94C014D45B4B707BD
:104F500010F023A0A7F201A03971130341022ED251
:104F60009A8506CE32D436D63AD83EDA42DC46DED0
:104F70001AC62D32F2400145216182805D71130312
:104F8000810322D42AC632DC2A841A86680006D617
:104F9000BEC236DEBAC0C2C4C6C61ACEEFF04FD407
:104FA000B247238007003245B250018D225461611F
:104FB0008280B70710F083A647F403A607F403A77F
:104FC00047F4E31AD7FE8966938606F4B29633B6A1
:104FD000C600B305E60023A4D7F423A6B7F4828065
:104FE000B70710F003A747F403A607F483A647F416
:104FF000E31AD7FE8966938606F4B29633B6C600E6
:1050000023A4D7F4B305E60023A6B7F4930700085A
:1050100073A047308280411122C406C697B70100B1
:105020009387074E17B401001304444D98431C4066
:105030001306F07C930647069387470697B5010051
:1050400023A0D54C97B5010023AAF54A6346D600A4
:10505000B2402244410182801307478997B701007B
:1050600023A0E74A2D2D85476310F5021840856778
:105070009387F7760145E3DDE7FCEFF05FED22442F
:10508000B24041016FC07FEC17B501001305053434
:10509000EFF09FEC0945EFF09FEB2244B240410155
:1050A0006FC0BFEA17B50100130505346FF0DFEAE2
:1050B00017B501001305C5336FF01FEA411122C473
:1050C00026C206C6856417B401001304E432938730
:1050D00084380100FD17F5FF2285EFF0FFE7C5BF1B
:1050E0000145EDA1411106C65D2B054781476316B9
:1050F000E500B2403E854101828017B501001305ED
:10510000E52CEFF07FE5B24089473E854101828082
:105110007370043001A082807370043001A04111CB
:1051200022C406C617B401001304C43E0145EFD0E3
:105130003F931C40850717B70100232DF73CFDB7AF
:10514000411122C426C206C6AA8405440145EFD0F7
:105150003F9181467D5681452685EFB05FAB814604
:105160000146814563008502268597B7010023A982
:10517000873AEFB09F96E30B85FC97B7010023A118
:10518000873AE9B78146014681452685EFB0FF940D
:10519000E30E85FA97B7010023A4873845BF0111B4
:1051A00022CC26CA4AC84EC652C456C25AC006CEDF
:1051B000AA8917BB0100130BAB3597BA0100938A7C
:1051C000EA3417B901001309E93417BA0100130AC8
:1051D000AA3405448D448146014681454E85EFB091
:1051E0001FA36306850097B7010023AB87320145F3
:1051F00097B7010023A00732EFC0CFFD09C597B7CD
:10520000010023AF873003250B00EFC01F97014536
:10521000EFC04FFC6306950097B7010023A28730CB
:1052200001458545EFC05F830145EFC0AFFA6306D6
:10523000950097B7010023A5872E03A50A00EFC0AC
:10524000DF938327090089C797B7010023AA872C1A
:105250008146014681454E85EFB03F886306850053
:1052600097B7010023AE872A83270900638687004A
:1052700097B7010023A6872A0145EFC0AFF5630663
:10528000850097B7010023AD872881450145EFC010
:10529000AFFC83270A00850717B70100232EF726E6
:1052A0001DBF397152D417BA0100130A2A2722DC14
:1052B00026DA4AD84ED656D25AD05ECE06DE62CC18
:1052C0002A84D28B094B9144954A2D4999498546A8
:1052D0000146DE852285EFB05F802285EFB09FF624
:1052E00085476306F50017B70100232BF722814697
:1052F00001462C002285EFB09F9185476306F5009B
:1053000017B70100232EF72003270A00A2476307DF
:10531000F700854717B701002324F7202285EFB057
:105320007FF211C5854717B70100232BF71E814671
:105330000146DE852285EFB04FFA2285EFB09FF05F
:1053400085476306F50017B70100232BF71C81463C
:1053500001462C002285EFB09F8B85476306F50040
:1053600017B70100232EF71A2285EFB0BFED11C544
:10537000854717B701002325F71A03270A00A2471C
:105380006307F700854717B70100232BF7185AC4A6
:10539000814601462C002285EFB02FF4A2478507F5
:1053A0003EC4E3F7F4FE2285EFB0DFE98D476307E3
:1053B000F500854717B701002324F71685460146F7
:1053C0002C00054C228562C4EFB02FF185460146C2
:1053D0002C00228502C4EFB04FF02285EFB09FE68B
:1053E0006306550197B7010023AC87138546014634
:1053F0002C002285EFB06FEE11C5854717B701006D
:105400002320F712814601462C002285EFB0EFECF5
:1054100011C5854717B701002324F71002C485463C
:1054200001466C002285EFB08FFE8547814601461C
:105430006C006306F50017B701002323F70EB2478F
:105440002248228513C7F7FF6307F800854717B87E
:1054500001002327F80C3AC6EFB06FFB85476306BF
:10546000F50017B70100232DF70AA247B2461387AC
:1054700017006388D714854797B6010023A2F60A60
:105480003AC4E3FEE4F82285EFB0DFDB11C58547BF
:1054900017B701002326F708A947814601462C00CB
:1054A00022853EC4EFB06FE385476306F50017B76A
:1054B00001002327F706814601462C0022854AC4B5
:1054C000EFB0AFE185476306F50017B70100232968
:1054D000F7042285EFB01FD763076501854717B72B
:1054E0000100232FF702A5473EC4854601462C0044
:1054F0002285EFB08FDE8547630FF50A17B70100ED
:105500002320F702A247FD173EC4E3E0F9FE2285FF
:10551000EFB05FD363075501854717B7010023211B
:10552000F700854601462C002285EFB00FDB11C540
:10553000854717B701002325F7FE814601462C0059
:105540002285EFB08FD911C5854717B701002329F0
:10555000F7FC9D473EC4054C814601466C00228500
:10556000EFB0EFEA6306850197B7010023AA87FB36
:10557000A247B24613871700638AD70297B7010084
:1055800023A087FB3AC4E379E9FC2285EFB09FCBE7
:1055900011C5854717B701002324F7F883270A00B0
:1055A000850717B70100232BF7F615B385073EC40F
:1055B000E374F9FAD9BFA247FD173EC4E3E7F9F255
:1055C000B9B785073EC4E3FCF4E475BD411126C2BA
:1055D0000146AA849145154506C622C4EFB00F8E38
:1055E00097B50100938585E22A84EFB03FD52687E1
:1055F000A2868148014881471306004097B5010003
:10560000938505E2170500001305E5C9EFB07FEBB0
:105610000545EFB06FC297B501009385E5E02A8498
:10562000EFB0DFD1A28681480148814701471306C8
:10563000004097B501009385E5DF170500001305CD
:1056400045B6EFB01FE88148014897B7010093873E
:10565000E7EB094781461306004097B501009385A3
:10566000E5DD170500001305C5ABEFB09FE5A28689
:105670002244B24092448148014897B70100938781
:1056800027E90D471306004097B50100938585DB98
:1056900017050000130505AB41016FB09FE217B776
:1056A00001001307A7E797B601009386E6E51C43C0
:1056B00094426397F600854797B6010023A2F6E669
:1056C00097B70100938747E517B60100130686E3F5
:1056D000944310426304D60297B60100938646E4D1
:1056E000184388429C4397B6010023AFE6E0133588
:1056F000150017B701002327F7E0828018439C4369
:10570000854617B60100232DD6E0014597B6010066
:1057100023ACE6DE17B701002326F7DE8280AA95C8
:10572000AA876385B70003C7070001E73385A74051
:1057300082808507FDB7814863DA05003305A04004
:10574000B337A000B305B0409D8DFD5863D9060066
:105750003306C040B337C000B306D0409D8E3288B8
:105760003683AA872E87639F061C97B6010093860F
:1057700066B463F1C50C416E6377C60B130EF00F70
:105780006373CE002143335E6600F29603CE0600BB
:105790001A9E130300023303C341630C0300B39545
:1057A0006500335EC501331866003367BE00B3176A
:1057B0006500135E0801B355C70313150801418145
:1057C00093D607013376C703B305B5024206D18EDF
:1057D00063F8B600C29663E5060163F3B600C296AD
:1057E0008D8E33F7C603C207C183B3D6C603B30693
:1057F000D50213150701C98F63F8D700C29763E577
:10580000070163F3D700C297958F33D567008145B1
:10581000638A0800B307A0403337F000B305B040F7
:105820003E85998D8280370E00014143E36DC6F5B8
:10583000614391BF01E605483358680241676373CD
:10584000E8081307F00F637307012143335768001B
:10585000BA9603C606001A96130300023303C34028
:1058600063190306B3850541935608011315080112
:10587000418113D6070133F7D502B3D5D5024207CC
:10588000518FB305B5026378B7004297636507018E
:105890006373B7004297B305B74033F7D502C20729
:1058A000C183B3D5D502B305B50213150701C98F5E
:1058B00063F8B700C29763E5070163F3B700C297C7
:1058C0008D8FA1B7370700014143E361E8F86143D9
:1058D000B5BF3318680033DEC500935E0801335648
:1058E000C500B31765003355DE03B39565004D8ED3
:1058F00093150801C181935606013377DE03338582
:10590000A5024207558F6378A70042976365070198
:105910006373A7004297B306A74033F7D603420646
:105920004182B3D6D6034207B386D502B365C7001A
:1059300063F8D500C29563E5050163F3D500C29510
:10594000958D1DB7E3E6D5EC416863F50605930E2A
:10595000F00F33B8DE000E0833DE060117B3010086
:10596000130343957293834E0300130E0002C29EED
:10597000330EDE4163170E0263E4B6006369C500AF
:10598000B307C540958D3335F5003387A5403E8577
:10599000BA85BDBD370300014148E3EF66FA6148AF
:1059A00065BF3357D601B396C601D98EB357D5011B
:1059B00033D7D501B395C501CD8F93D50601337388
:1059C000B702139F0601135F0F0113D807013316A7
:1059D000C6013315C5013357B702420333680301CB
:1059E000B30FEF023A83637CF80136981303F7FF95
:1059F0006367D8006375F8011303E7FF369833082F
:105A0000F841B37FB8023358B802C20FB3050F0391
:105A1000139F0701135F0F0133EFEF014287637C90
:105A2000BF00369F1307F8FF6367DF006375BF0091
:105A30001307E8FF369F4203C16F3363E300938788
:105A4000FFFF13580601330FBF40B375F300135324
:105A50000301F18F3387F502B307F302B385050322
:105A600033030303BE95135807012E986373F800A0
:105A70007E93C167FD17935508013378F8004208FB
:105A80007D8F9A9542976366BF00631BBF00637961
:105A9000E5003306C7403337C700958D998D3287AF
:105AA0003307E5403335E500B305BF40898DB39733
:105AB000D5013357C70133E5E700B3D5C50189BB2D
:105AC000AE87328836872A836396062097A801001E
:105AD0009388487E63FEC50A41676374E60A13072C
:105AE000F00F3337C7000E07B356E600B69883C6EB
:105AF0000800369793060002998E99CAB397D7008B
:105B00003357E5003318D600B365F7003313D500DB
:105B100013550801B3D7A502131608014182935605
:105B2000030133F7A502B305F6024207D98E3E877B
:105B300063FCB600C2961387F7FF63E7060163F5BF
:105B4000B6001387E7FFC2968D8EB3F7A602420315
:105B500013530301B3D6A602C20733E36700B305AC
:105B6000D6023685637BB30042931385F6FF6366E6
:105B700003016374B3001385E6FF4207498F814533
:105B80004DA8B70600014147E360D6F66147A9BFBB
:105B900001E6854633D8C602C166637ED8089306FF
:105BA000F00F63F306012147B356E800B69883C6A9
:105BB0000800BA9613070002158F49E7B38707411B
:105BC0008545135608019318080193D80801935688
:105BD000030133F7C702B3D7C7024207D98E338513
:105BE000F8023E8763FCA600C2961387F7FF63E7BF
:105BF000060163F5A6001387E7FFC296898EB3F707
:105C0000C602420313530301B3D6C602C20733E3ED
:105C10006700B388D8023685637B130142931385EE
:105C2000F6FF63660301637413011385E6FF420701
:105C3000498F3A858280B70600014147E366D8F66E
:105C400061479DB73318E800B3D5D7003313E5009B
:105C5000B356D50013550801B397E70033F7A502F3
:105C6000B3E8F60093170801C18313D60801B3D532
:105C7000A5024207518FB386B7022E86637CD700F8
:105C800042971386F5FF636707016375D700138694
:105C9000E5FF4297B306D74033F7A602C20893D870
:105CA0000801B3D6A6024207B385D702B36717012E
:105CB000368763FCB700C2971387F6FF63E70701D7
:105CC00063F5B7001387E6FFC2978D8F9315060122
:105CD000D98DC5BD63E2D514416763FEE6021308A2
:105CE000F00F3337D8000E0733D8E60097A5010030
:105CF0009385455CC29503C80500930500023A9858
:105D0000B385054185E10547E3E5F6F23335C50086
:105D10001347150039BFB70500014147E3E6B6FC5C
:105D20006147D9B733570601B396B600D98E93DED3
:105D3000060133D70701B378D703B397B7003358B9
:105D400005013363F80093970601C18313580301DB
:105D50003316B6003357D703C20833E80801338F30
:105D6000E7023A8E637CE8013698130EF7FF63670B
:105D7000D8006375E801130EE7FF36983308E84151
:105D8000B378D8033358D803C208B38E07039317E8
:105D90000301C183B3E7F800428763FCD701B697DC
:105DA0001307F8FF63E7D70063F5D7011307E8FF90
:105DB000B697420EB387D741C16E3367EE001388A2
:105DC000FEFF3373070193580701337806014182C0
:105DD000330E03033388080393560E013303C302C3
:105DE00042939A96B388C80263F30601F69813D6D5
:105DF0000601B29863E01703E39317D9C167FD1753
:105E0000FD8EC206337EFE003315B500F296814545
:105E1000E371D5E27D17A5B38145014719BDB2886D
:105E20003687AA872E886398061C97A6010093865A
:105E3000664863F8C50A4163637E66081303F00F82
:105E40006373C30021473353E6009A9603CE0600DE
:105E5000130300023A9E3303C341630C0300B3955E
:105E60006500335EC501B31866003368BE00B31722
:105E7000650013D608013377C802139508014181E4
:105E800093D607013358C8024207D98E3308050359
:105E900063F80601C69663E5160163F30601C6962C
:105EA000B386064133F7C602C207C183B3D6C60222
:105EB000B306D50213150701C98F63F8D700C6973B
:105EC00063E5170163F3D700C697958F33D5670055
:105ED00081458280370300014147E36666F66147EA
:105EE0009DB701E60546B3581603416663F3C8083B
:105EF0001306F00F63731601214733D6E800B296FC
:105F000003CE0600130300023A9E3303C341631914
:105F10000306B385154113D7080113950801418184
:105F200013D60701B3F6E502B3D5E502C206D18E5A
:105F3000B305B50263F8B600C69663E5160163F3D0
:105F4000B600C696B385B640B3F6E502C207C18374
:105F5000B3D5E502B305B50213950601C98F63F801
:105F6000B700C69763E5170163F3B700C6978D8F37
:105F7000B1BF370600014147E3E1C8F86147B5BF4B
:105F8000B398680033D7C501B3176500335EC50108
:105F900013D50801B376A702B3956500336EBE0032
:105FA00093950801C18113560E013357A702C2060B
:105FB000D18E3387E50263F8E600C69663E51601E5
:105FC00063F3E600C6963386E640B376A602420E39
:105FD000135E0E013356A602C2063386C502B3E530
:105FE000C60163F8C500C69563E5150163F3C500F6
:105FF000C695918D0DB7E3EED5EC416763F5E604E8
:10600000930EF00F33B7DE000E0733D3E60097A8E8
:1060100001009388282A9A9883CE0800130E000264
:10602000BA9E330EDE4163170E0263E4B600636965
:10603000C500B307C540958D3335F5003388A540BD
:106040003E85C28579B5B70800014147E3EF16FBED
:10605000614765BF3357D601B396C601D98EB35792
:10606000D50133D7D501B395C501CD8F93D50601A1
:106070003373B702139F0601135F0F0193D8070113
:106080003316C6013315C5013357B7024203B3684F
:1060900013013308EF023A8363FC0801B698130337
:1060A000F7FF63E7D80063F508011303E7FFB6982D
:1060B000B3880841B3FFB802B3D8B802C20FB30522
:1060C0001F03139F0701135F0F0133EFEF01468793
:1060D000637CBF00369F1387F8FF6367DF0063753B
:1060E000BF001387E8FF369F4203C1683363E300B4
:1060F0009387F8FF13580601330FBF40B375F300C1
:1061000013530301F18F3387F502B307F302B3850D
:10611000050333030303BE95135807012E986373D9
:10612000F8004693C167FD17935508013378F800CE
:1061300042087D8F9A9542976366BF00631BBF003C
:106140006379E5003306C7403337C700958D998DD5
:1061500032873307E5403335E500B305BF40898D0D
:10616000B397D5013357C70133E5E700B3D5C50170
:106170008DB397A701009387A735944317A7010014
:106180001307C7331843C8C2637BE50017A7010094
:106190001307873308438C4391056FA06FBA4111F1
:1061A00022C406C617A70100130747322A840843F2
:1061B0008C439105EFA0CFB897A701009387472E96
:1061C0009C436376F40097A7010023AB872CB24071
:1061D00022444101828097A701009387672F98434B
:1061E00094437C43FD177CC3FC4299E37360043005
:1061F0008280011122CC26CA2A84AE844AC84EC6A7
:1062000052C456C206CEEFB05FD51C40032904012C
:10621000B7090001B3E59700930AC4000CC081449C
:10622000FD19370A00021840638C2A03032609006F
:106230004A85B3654701B376360193175600758FCB
:106240000329490063C4070001E7F1BFE39DE6FCB1
:106250009317760063D30700D58CEFC0FFBEE1B77C
:1062600093C4F4FFF98C04C0EFB03FF40840F2404F
:106270006244D2444249B249224A924A056182802C
:106280004111014506C622C4EFF04FB417F7FFFFD6
:106290001307A7D8814605469305200317A50100DB
:1062A00013050516EFD05F8E19C92A84EFB0FFCB16
:1062B0002A860147814685452285EFD09F99EFB018
:0C62C0005FA4B2402244014541018280ED
:02000004800278
:100000001247FEFF1048FEFF1A47FEFF1048FEFF92
:100010001048FEFF1048FEFF1048FEFF3247FEFF6B
:100020001048FEFF1048FEFF4C47FEFF5847FEFFFA
:100030001048FEFF6A47FEFF7647FEFF7647FEFF49
:100040007647FEFF7647FEFF7647FEFF7647FEFFC8
:100050007647FEFF7647FEFF7647FEFF1048FEFF1D
:100060001048FEFF1048FEFF1048FEFF1048FEFF3C
:100070001048FEFF1048FEFF1048FEFF1048FEFF2C
:100080001048FEFF1048FEFF1048FEFF1048FEFF1C
:100090001048FEFF1048FEFF1048FEFF1048FEFF0C
:1000A0001048FEFF1048FEFF1048FEFF1048FEFFFC
:1000B0001048FEFF1048FEFF1048FEFF1048FEFFEC
:1000C0001048FEFF1048FEFF1048FEFF1048FEFFDC
:1000D0001048FEFF1048FEFF1048FEFF1048FEFFCC
:1000E0001048FEFF1048FEFF1048FEFF1048FEFFBC
:1000F0001048FEFF1048FEFF1048FEFF1048FEFFAC
:10010000AA47FEFFC047FEFF1048FEFF1048FEFF53
:100110001048FEFF1048FEFF1048FEFF1048FEFF8B
:100120001048FEFF0648FEFF1048FEFF1048FEFF85
:10013000B845FEFF7046FEFF1048FEFF1048FEFF68
:10014000A646FEFF1048FEFFFE46FEFF1048FEFFDB
:100150001048FEFF2C47FEFF1E4BFEFF724BFEFFBA
:10016000264BFEFF724BFEFF724BFEFF724BFEFFF3
:10017000724BFEFF184AFEFF724BFEFF724BFEFFF2
:10018000324AFEFF3E4AFEFF724BFEFF504AFEFF20
:100190005C4AFEFF5C4AFEFF5C4AFEFF5C4AFEFFD3
:1001A0005C4AFEFF5C4AFEFF5C4AFEFF5C4AFEFFC3
:1001B0005C4AFEFF724BFEFF724BFEFF724BFEFF6E
:1001C000724BFEFF724BFEFF724BFEFF724BFEFF47
:1001D000724BFEFF724BFEFF724BFEFF724BFEFF37
:1001E000724BFEFF724BFEFF724BFEFF724BFEFF27
:1001F000724BFEFF724BFEFF724BFEFF724BFEFF17
:10020000724BFEFF724BFEFF724BFEFF724BFEFF06
:10021000724BFEFF724BFEFF724BFEFF724BFEFFF6
:10022000724BFEFF724BFEFF724BFEFF724BFEFFE6
:10023000724BFEFF724BFEFF724BFEFF724BFEFFD6
:10024000724BFEFF724BFEFF724BFEFF724BFEFFC6
:10025000724BFEFF724BFEFF904AFEFFBE4AFEFF4E
:10026000724BFEFF724BFEFF724BFEFF724BFEFFA6
:10027000724BFEFF724BFEFF724BFEFF144BFEFFF4
:10028000724BFEFF724BFEFF7648FEFF7049FEFF89
:10029000724BFEFF724BFEFFE249FEFF724BFEFF08
:1002A000084AFEFF724BFEFF724BFEFF6C4BFEFFD7
:1002B000000102020303030304040404040404040D
:1002C00005050505050505050505050505050505DE
:1002D00006060606060606060606060606060606BE
:1002E00006060606060606060606060606060606AE
:1002F000070707070707070707070707070707078E
:10030000070707070707070707070707070707077D
:10031000070707070707070707070707070707076D
:10032000070707070707070707070707070707075D
:10033000080808080808080808080808080808083D
:10034000080808080808080808080808080808082D
:10035000080808080808080808080808080808081D
:10036000080808080808080808080808080808080D
:1003700008080808080808080808080808080808FD
:1003800008080808080808080808080808080808ED
:1003900008080808080808080808080808080808DD
:1003A00008080808080808080808080808080808CD
:1003B000546D725100000000546D7220537663003A
:1003C000286E756C6C2900004572726F7220696E20
:1003D00020416C745154657374207461736B732085
:1003E0000D0A00006D69616F750A00006D69616F2B
:1003F00075320A0068756E6772790A004368656332
:100400006B54696D65720000416C745F47656E5F87
:10041000546573745F517565756500004647656E78
:1004200051000000416C745F515F4D757465780038
:10043000464D754C6F770000464D754D6564000064
:08044000464D7548696768002C
:100448001000000000000000017A5200017C010148
:100458001B0D02001000000018000000D252FEFF21
:100468008A03000000000000100000002C000000BB
:100478004856FEFF5E030000000000001000000068
:10048800400000009259FEFF5403000000000000E5
:08052000FC8F0100090000003E
:040000058000004037
:00000001FF
